:04000000BFEF02F05C
:1000080000C016F001C015F0E1CF17F0E2CF18F0EC
:100018009DAA74D09EAA72D0AECF1FF0ABA40DD00B
:10002800AB9E010E4724006E000E4820016E00C0F2
:1000380047F001C048F0AB8E1F6AABA20DD0AB9859
:10004800AB88010E4524006E000E4620016E00C0EC
:1000580045F001C046F01F6A000E0001A41902E134
:10006800010EA31917E1A50EA125E16E000EA2212C
:10007800E26EE66A010E0101A96F000EAA6FA1C027
:10008800A7F1A2C0A8F10001A16BA26BAECF1FF02F
:100098009D9A16D0A50EA125E16E000EA221E26E52
:1000A8001FC0E6FF010EA125006E000EA221016E01
:1000B80000C0A1F001C0A2F0A1C0A7F1A2C0A8F1A0
:1000C800800E010A006E800EA219005C02E1A151A7
:1000D800000814E2020E0101A96F000EAA6F9D9A92
:1000E800020E0001A15D006E000EA259016EA50E60
:1000F8000024E16E000E0120E26EE66A9DA020D089
:100108009EA01ED0010E0101C15D006E000EC259F5
:10011800016E00C0C1F101C0C2F1000EC25D02E172
:10012800010EC15D08E2C16BC26B010E0001A36F35
:10013800000EA46F9D903C0ECF6EB00ECE6E9E90BA
:1001480016C000F015C001F017C0E1FF18C0E2FFAB
:02015800110094
:10015A000101CC1D206E080E216E8994C9EC00F0B5
:10016A002032D8B0BCEF00F08984BDEF00F089944A
:10017A00C9EC00F0212EB5EF00F08984C9EC00F03B
:10018A00C9EC00F0D6EF00F01C0E226E0000000051
:10019A0000000000222ECBEF00F00000000000005B
:0601AA001200000012002B
:1001B000CBC100F00101CB07005228E0C7C1E9FF25
:1001C000C8C1EAFFEE50000A0CE0C7C1E9FFC8C190
:1001D000EAFFC9C1D9FFCAC1DAFFEE50DE1801E15A
:1001E0000FD0C7C1E9FFC8C1EAFFC9C1D9FFCAC161
:1001F000DAFFDE50EE5C006E016A000E015A08D094
:100200000101C74BC82BC94BCA2BD2D7006A016A60
:020210001200DA
:10021200C7C102F0C8C103F002C000F003C001F080
:10022200024A032A00C0E9FF01C0EAFFEE5201E0E0
:10023200F3D70101C751025C006EC8510358016E29
:0A024200010E005E000E015A1200CA
:10024C00C7C1E9FFC8C1EAFFEE500101C91905E1B8
:10025C00C7C100F0C8C101F010D0C7C100F0C8C1BF
:10026C0001F0C74BC82B00C0E9FF01C0EAFFEECF7D
:0C027C0000F00052E5E1006A016A120087
:10028800C7C1F6FFC8C1F7FFC9C1F8FF0900F5CF1C
:1002980000F0005210E0C7C1F6FFC8C1F7FFC9C19E
:1002A800F8FF0900F5CFCCF154DF010EC727000E87
:0802B800C823C923E5D7120099
:1002C0000B6A0A6A096A00500402F4CF09F0F3CFFE
:1002D00008F001500502F4CF0BF0F3CF0AF0005004
:1002E0000502F3500926F4500A22E86A0B22015055
:1002F0000402F3500926F4500A22E86A0B2208C0CF
:1003000000F009C001F00AC002F00BC003F01200B7
:0E031000ACB202D00000FCD7C7C1ADFF120096
:10031E000900F5CFE6FF0006FBE10106F9E1120048
:10032E00806A0F01386B3881230E926E92988988FD
:10033E009296898692948984396BFF0E816E8F0E08
:10034E00936EF19E3A6B826AFF0E946E949C949219
:08035E0094908B80606A12008C
:10036600100E0101B36F030EB46FC70EB56F010E09
:10037600B66FFF0EB76FFF0EB86F000EB96F000EA7
:10038600BA6FFF0EAB6FFF0EAC6F000EAD6F000EB7
:10039600AE6FFF0EAF6FFF0EB06F000EB16F000EA7
:1003A600B26FAC8A900EAB6E948E949C9EAA03D0CC
:0803B600AECF00F0FBD71200EE
:1003BE00000E0101C41902E1000EC31934E0C3C1DD
:1003CE00E9FFC4C1EAFFEE522EE0C5C1C7F1C6C1B6
:1003DE00C8F118DF00C0CBF1C3C1C7F1C4C1C8F169
:1003EE00C5C1C9F1C6C1CAF1DCDE000E011802E1B9
:1003FE00000E001805E1C3C100F0C4C101F015D014
:10040E00010E0101C325C76F000EC421C86FC5C1FF
:10041E00E9FFC6C1EAFFEECFC9F111DF00C0C3F19B
:0C042E0001C0C4F1C5D7006A016A1200C9
:10043A00016A026A800E0218006E800E000A005CD1
:10044A0002E1FF0E015C0AE2A50E0124E16E000E34
:10045A000220E26EE66A014A022AECD7AECF1FF00A
:10046A000001A56B1F6AA16BA26B0101A76BA86BA8
:08047A00A96BAA6B9D8A120018
:10048200C3C1F6FFC4C1F7FFC5C1F8FF0900F5CF2C
:1004920000F0005211E0C3C1F6FFC4C1F7FFC5C1AD
:1004A200F8FF0900F5CFC7F132DF010E0101C327C2
:0A04B200000EC423C523E4D7120096
:1004BC000D0E0101CC6F4BDE0A0ECC6F48DE120024
:1004CC000101A56BA66B800EA619006E800E005C58
:1004DC0002E10A0EA55D27E2030E006E000E016E0E
:1004EC00A5C104F0A6C105F0E5DE240E0024E96EDA
:1004FC00000E0120EA6EEECFC7F1EECFC8F1EECFC1
:10050C00C9F1BCDE070E0B6E170E0C6E6A0E0D6E6B
:10051C000D2EFED70C2EFCD70B2EFAD700000101A6
:08052C00A54BA62BD0D712004D
:10053400C3C1E9FFC4C1EAFFEE5000080AE2C3C127
:10054400E9FFC4C1EAFFEECFCCF105DEC34BC42BF7
:04055400EFD71200CB
:10055800300ECD6E9E903C0ECF6EB00ECE6EC3C1E7
:10056800C1F1C4C1C2F10001A36BA46B9E909D9020
:06057800CD809D80120001
:10057E00E5EC05F09B6A720ED36E9B9CD26AD3B4E7
:10058E0001D0FDD7CDDE206A216A226A236A8FDF71
:10059E00A56BA66B800EA619006E800E005C02E1A4
:1005AE00040EA55D21E289968988070E0B6E170E43
:1005BE000C6E6A0E0D6E0D2EFED70C2EFCD70B2E6A
:1005CE00FAD7000089868998070E0B6E170E0C6EEF
:1005DE006A0E0D6E0D2EFED70C2EFCD70B2EFAD7F3
:1005EE000000A54BA62BD6D789868998496A4A6AF8
:1005FE00456A466A476A486A00019D6B9E6BAB6A04
:10060E00AB88AB8EAB8A9F6BA06B70821F6A89988A
:10061E004D0E4B6E000E4C6E52DF899448DFB8863D
:10062E00010EB06EA00EAF6EAC8496DE050E0B6E94
:10063E000F0E0C6EF10E0D6E0D2EFED70C2EFCD77E
:10064E000B2EFAD79D809D8AF28CF28EA70EC76F65
:10065E000A0EC86F000EC96F10DE8B900B0E0B6E5C
:10066E00260E0C6E5D0E0D6E0D2EFED70C2EFCD7CB
:10067E000B2EFAD700000000910E0101C36F0B0E76
:10068E00C46F000EC56FF6DE9C0E0101C36F0B0E1C
:10069E00C46F000EC56FEEDE030E0B6E080E0C6EF1
:1006AE00770E0D6E0D2EFED70C2EFCD70B2EFAD715
:1006BE00A60E0101C36F0B0EC46F000EC56FDADEFE
:1006CE00030E0B6E080E0C6E770E0D6E0D2EFED7F2
:1006DE000C2EFCD70B2EFAD7DE0E0101C76F090EBA
:1006EE00C86F000EC96FC9DDAF0E0101C76F0B0ECB
:1006FE00C86F000EC96FC1DD99DE140EC36F000EF8
:10070E00C46F23DFB70E0101C36F0B0EC46F000E53
:10071E00C56FB0DE050E0B6E0F0E0C6EF10E0D6E6C
:10072E000D2EFED70C2EFCD70B2EFAD7000E000185
:10073E00A41902E1000EA31908E1000E0101AA1985
:10074E0002E1000EA91901E1F1D70001A36BA46B20
:10075E00000E0101AA1902E1010EA9190AE0800E8C
:10076E00006E800EA819005C02E1A751020801E399
:10077E000CD00001A36BA46B9ADEA50EC36F000E06
:10078E00C46FD1DE94DEAECF1FF08B800B0E0B6EDE
:10079E00260E0C6E5D0E0D6E0D2EFED70C2EFCD79A
:1007AE000B2EFAD700000000BB6BBC6BBD6BBE6B93
:1007BE001E6A8B80030E0B6E080E0C6E770E0D6E7E
:1007CE000D2EFED70C2EFCD70B2EFAD7B886010EA7
:1007DE00B06EA00EAF6EAC84BFDDC50EC76F0B0E34
:1007EE00C86F000EC96F49DD320E0101C36F000ED6
:1007FE00C46FABDE1BDE810EC36F0B0EC46F000E1B
:10080E00C56F38DE000E0001A41902E1000EA31917
:10081E0008E1000E0101AA1902E1000EA91901E179
:10082E00F1D70101000EAA1902E1010EA9190AE081
:10083E00800E006E800EA819005C02E1A75105081B
:10084E0001E321D0A50EC36F000EC46F190EC56F44
:10085E00000EC66FADDD00C0BFF101C0C0F1000ECD
:10086E00026E0150025C02E1005000080BE2000132
:10087E00E56BAA0E0101C36F000EC46F54DE0101B9
:10088E00BF6BC06B01D013DE0101000EAA1902E18D
:10089E00020EA9190AE1370EC76F0B0EC86F000EB4
:1008AE00C96FEBDC0101A96BAA6BBB4BBC2B95D7B7
:0208BE00FFD762
:100BCA0010EE24F0210E006E010E016E160EF66E66
:100BDA000B0EF76E000EF86E8FEC01F010EE19F0A6
:100BEA00060E006E010E016EBF0EF66E0B0EF76E4C
:0A0BFA00000EF86E8FEC01F01200FF
:1008C0002050726F6A6574203A20503138463236B3
:1008D0004B32325F436F6E63656E7472617465751F
:1008E000725F5370656369616C5F484331325F6367
:1008F000616E616C5F31365F4655335F393630303B
:100900005F3139313031372E6D637070690D0A00F7
:1009100020536F75726365205031384632364B3242
:10092000325F436F6E63656E747261746575725F7A
:100930005370656369616C5F484331325F43616E38
:10094000616C31365F4655335F393630305F5F3129
:0A09500039313031372E630D0A00F3
:10095A00204469726563746F72793A20433A5C5F26
:10096A004D696B726F435C5F4D657350726F6A6558
:10097A0074735F4D696B726F435C5F484331325FDA
:10098A005472616E736365697665725F3433334D91
:05099A00687A0D0A005F
:10099F0020464F534320696E7465726E6520203177
:1009AF00364D487A20766961205031384632364BC1
:1009BF0032325F464F53435F696E7465726E655F87
:0F09CF0031364D687A2E6366677363680D0A00D0
:1009DE000D0A204C656374757265205365747469D5
:1009EE006E672020484331322073757220636F6E1C
:1009FE0063656E74726174657572204261736520F1
:0C0A0E0050494332364B32320D0A2000B2
:100A1A0020436F6E666967203A2050313846323675
:100A2A004B32325F464F53435F696E7465726E652F
:100A3A005F31364D687A2E6366677363680D0A0004
:100A4A0020506F72742048617264205541525431AB
:100A5A0020343830302C4E2C382C31202852433652
:0F0A6A003D5458205243373D525829200D0A0061
:100A79002041766563205458205541525433203122
:100A890039323030626473202041534D20737572BE
:0E0A990020524132206F75747075740D0A0082
:100AA70020496E69742053657474696E672020430A
:100AB700616E616C203136206D6F6465202046556C
:080AC7003320393630302000E5
:100ACF00205241303D41444320205241313D4F5748
:100ADF00532073656E736F72204453313842323036
:040AEF00200D0A00CC
:100AF300204D435520203A31384632364B3232208E
:100B0300416C696D2E203D20342E3520E020355672
:030B13000D0A00C8
:100B16005A0900C00800F30A001A0A009F09004A91
:100B26000A00CF0A00100900790A006A0B00520B6E
:010B360000BE
:100B3700205042206465626F7264656D656E742033
:0B0B470062756666657231200D0A00C1
:100B5200204C616E67616765204D696B726F43203F
:080B6200372E3530200D0A008A
:100B6A0020454550524F4D206E6F6E207574696C4A
:070B7A006973E9650D0A0033
:100B810057616974696E67206D736720210D0A00D2
:0B0B910041542B42393630300D0A0071
:0A0B9C0041542B433031360D0A009E
:090BA60041542B4655330D0A00A1
:080BAF0041542B52580D0A00BD
:080BB70041542B52580D0A00B5
:050BBF004B4D4C2C0021
:010BC4000030
:050BC5004B4D4C2C001B
:020000040030CA
:0D000100281F3CFFBF81FF0FC00FE00F4024
:00000001FF
